 nessus

 Timestamp is 3a0abb41 (Thu Nov 09 15:57:05 2000)

 Preferred load address is 00400000

 Start         Length     Name                   Class
 0001:00000000 0002155cH .text                   CODE
 0002:00000000 0000046cH .idata$5                DATA
 0002:00000470 000000bcH .rdata                  DATA
 0002:0000052c 000000a0H .idata$2                DATA
 0002:000005cc 00000014H .idata$3                DATA
 0002:000005e0 0000046cH .idata$4                DATA
 0002:00000a4c 00000f9cH .idata$6                DATA
 0002:000019e8 00000000H .edata                  DATA
 0003:00000000 00000004H .CRT$XCA                DATA
 0003:00000004 00000004H .CRT$XCZ                DATA
 0003:00000008 00000004H .CRT$XIA                DATA
 0003:0000000c 00000004H .CRT$XIZ                DATA
 0003:00000010 00097724H .data                   DATA
 0003:00097734 000108c8H .bss                    DATA

  Address         Publics by Value              Rva+Base     Lib:Object

 0001:00000000       _attack_host               00401000 f   attack.obj
 0001:000002a0       _auth_login                004012a0 f   auth.obj
 0001:00000380       _network_printf            00401380 f   auth.obj
 0001:00000400       _network_gets              00401400 f   auth.obj
 0001:00000440       _network_gets_raw          00401440 f   auth.obj
 0001:00000510       _comm_init                 00401510 f   comm.obj
 0001:00000590       _comm_get_preferences      00401590 f   comm.obj
 0001:00000920       _comm_send_preferences     00401920 f   comm.obj
 0001:00000c60       _comm_send_rules           00401c60 f   comm.obj
 0001:00000cc0       _comm_get_preferences_errors 00401cc0 f   comm.obj
 0001:00000d00       _comm_get_rules            00401d00 f   comm.obj
 0001:00000e00       _comm_get_pluginlist       00401e00 f   comm.obj
 0001:000012c0       _comm_server_restores_sessions 004022c0 f   comm.obj
 0001:000012d0       _comm_get_sessions         004022d0 f   comm.obj
 0001:000013f0       _comm_delete_session       004023f0 f   comm.obj
 0001:00001410       _comm_restore_session      00402410 f   comm.obj
 0001:00001430       _show_dialog               00402430 f   error_dialog.obj
 0001:00001710       _show_dialog_and_wait_build 00402710 f   error_dialog.obj
 0001:00001a10       _show_dialog_and_wait      00402a10 f   error_dialog.obj
 0001:00001a80       _family_init               00402a80 f   families.obj
 0001:00001a90       _family_add                00402a90 f   families.obj
 0001:00001b50       _family_enable             00402b50 f   families.obj
 0001:00001c20       _family_enabled            00402c20 f   families.obj
 0001:00001ca0       _monitor_dialog_setup      00402ca0 f   monitor_dialog.obj
 0001:00001f80       _monitor_remove_host       00402f80 f   monitor_dialog.obj
 0001:00002f40       _log_write                 00403f40 f   nessus.obj
 0001:00002f60       _connect_to_nessusd        00403f60 f   nessus.obj
 0001:00003330       _init_globals              00404330 f   nessus.obj
 0001:00003370       _display_help              00404370 f   nessus.obj
 0001:000033c0       _main                      004043c0 f   nessus.obj
 0001:00003e70       _WinMain@16                00404e70 f   nessus.obj
 0001:00003eb0       _parse_message_type        00404eb0 f   parser.obj
 0001:00004150       _parse_server_message      00405150 f   parser.obj
 0001:00004430       _parse_nessusd_status      00405430 f   parser.obj
 0001:00004510       _parse_host_add_port       00405510 f   parser.obj
 0001:00004660       _parse_host_add_data       00405660 f   parser.obj
 0001:00004c70       _parse_symbol              00405c70 f   parser.obj
 0001:00004cb0       _parse_separator           00405cb0 f   parser.obj
 0001:00004e90       _pass_dialog               00405e90 f   password_dialog.obj
 0001:000052f0       _keypass_dialog            004062f0 f   password_dialog.obj
 0001:00005370       _cmdline_pass              00406370 f   password_dialog.obj
 0001:00005380       _created_private_key       00406380 f   password_dialog.obj
 0001:00005390       _get_pwd                   00406390 f   password_dialog.obj
 0001:000054a0       _plugin_info_window_setup  004064a0 f   plugin_infos.obj
 0001:00005990       _preferences_init          00406990 f   preferences.obj
 0001:00005ab0       _preferences_process       00406ab0 f   preferences.obj
 0001:00006030       _preferences_save_fname    00407030 f   preferences.obj
 0001:00006200       _preferences_save          00407200 f   preferences.obj
 0001:00006220       _pluginset_apply           00407220 f   preferences.obj
 0001:00006330       _pluginset_reload          00407330 f   preferences.obj
 0001:00006560       _prefs_check_defaults      00407560 f   preferences.obj
 0001:00006570       _target_file_select        00407570 f   read_target_file.obj
 0001:000066c0       _target_file_to_list       004076c0 f   read_target_file.obj
 0001:00006920       _target_translate          00407920 f   read_target_file.obj
 0001:00006960       _target_file_name          00407960 f   read_target_file.obj
 0001:000069a0       _read_target_file          004079a0 f   read_target_file.obj
 0001:00006a50       _report_to_tree            00407a50 f   report.obj
 0001:000070c0       _is_there_any_hole         004080c0 f   report.obj
 0001:00007180       _report_tests              00408180 f   report.obj
 0001:00007fd0       _open_report               00408fd0 f   report.obj
 0001:00008010       _open_report_selectfile    00409010 f   report.obj
 0001:00008580       _latex_introduction_a      00409580 f   latex_output.obj
 0001:00008670       _latex_introduction_b      00409670 f   latex_output.obj
 0001:00008780       _latex_introduction_c      00409780 f   latex_output.obj
 0001:000088d0       _latex_introduction_d      004098d0 f   latex_output.obj
 0001:00008a20       _latex_introduction_e      00409a20 f   latex_output.obj
 0001:00008ba0       _latex_print_host_ports    00409ba0 f   latex_output.obj
 0001:00008bd0       _latex_print_host_ports_problems 00409bd0 f   latex_output.obj
 0001:00008de0       _latex_print_hosts         00409de0 f   latex_output.obj
 0001:00008ef0       _latex_conclusion          00409ef0 f   latex_output.obj
 0001:00009000       _latex_appendix_plugins    0040a000 f   latex_output.obj
 0001:00009060       _latex_appendix            0040a060 f   latex_output.obj
 0001:00009110       _arglist_to_latex          0040a110 f   latex_output.obj
 0001:00009390       _sighand_pipe              0040a390 f   sighand.obj
 0001:000093d0       _sighand_alarm             0040a3d0 f   sighand.obj
 0001:00009410       _sighand_exit              0040a410 f   sighand.obj
 0001:00009460       _init_display              0040a460 f   xstuff.obj
 0001:00009480       _close_window              0040a480 f   xstuff.obj
 0001:00009490       _delete_event              0040a490 f   xstuff.obj
 0001:000094a0       _close_display             0040a4a0 f   xstuff.obj
 0001:000094b0       _arglist_length            0040a4b0 f   report_utils.obj
 0001:000094d0       _sort_by_port              0040a4d0 f   report_utils.obj
 0001:00009890       _number_of_notes_by_port   0040a890 f   report_utils.obj
 0001:000098d0       _number_of_notes_by_host   0040a8d0 f   report_utils.obj
 0001:00009900       _number_of_warnings_by_port 0040a900 f   report_utils.obj
 0001:00009940       _number_of_warnings_by_host 0040a940 f   report_utils.obj
 0001:00009970       _number_of_holes_by_port   0040a970 f   report_utils.obj
 0001:000099b0       _number_of_holes_by_host   0040a9b0 f   report_utils.obj
 0001:000099e0       _number_of_notes           0040a9e0 f   report_utils.obj
 0001:00009a10       _number_of_warnings        0040aa10 f   report_utils.obj
 0001:00009a40       _number_of_holes           0040aa40 f   report_utils.obj
 0001:00009a70       _most_dangerous_host       0040aa70 f   report_utils.obj
 0001:00009ba0       _arglist_insert            0040aba0 f   report_utils.obj
 0001:00009c50       _arglist_insert_sort       0040ac50 f   report_utils.obj
 0001:00009c80       _sort_dangerous_hosts      0040ac80 f   report_utils.obj
 0001:00009cb0       _arglist_to_html           0040acb0 f   html_output.obj
 0001:0000a710       _arglist_to_file           0040b710 f   nsr_output.obj
 0001:0000aab0       _file_to_arglist           0040bab0 f   nsr_output.obj
 0001:0000afa0       _printf_formatted_text     0040bfa0 f   text_output.obj
 0001:0000b0d0       _arglist_to_text           0040c0d0 f   text_output.obj
 0001:0000b4f0       _splash_passphrase         0040c4f0 f   splash_screen.obj
 0001:0000bd60       _splash                    0040cd60 f   splash_screen.obj
 0001:0000c0b0       _arglist_to_html_graph     0040d0b0 f   html_graph_output.obj
 0001:0000df60       _cli_args_new              0040ef60 f   cli.obj
 0001:0000df70       _cli_args_server           0040ef70 f   cli.obj
 0001:0000dfa0       _cli_args_port             0040efa0 f   cli.obj
 0001:0000dfb0       _cli_args_login            0040efb0 f   cli.obj
 0001:0000dfe0       _cli_args_password         0040efe0 f   cli.obj
 0001:0000e010       _cli_args_target           0040f010 f   cli.obj
 0001:0000e040       _cli_args_results          0040f040 f   cli.obj
 0001:0000e0f0       _cli_args_cipher           0040f0f0 f   cli.obj
 0001:0000e120       _cli_args_auth_pwd         0040f120 f   cli.obj
 0001:0000e130       _cli_args_output           0040f130 f   cli.obj
 0001:0000e140       _cli_args_best_output      0040f140 f   cli.obj
 0001:0000e200       _cli_connect_to_nessusd    0040f200 f   cli.obj
 0001:0000e240       _cli_test_network          0040f240 f   cli.obj
 0001:0000e320       _cli_report                0040f320 f   cli.obj
 0001:0000e340       _arglist_to_xml            0040f340 f   xml_output.obj
 0001:0000eae0       _prefs_dialog_about        0040fae0 f   prefs_about.obj
 0001:0000ee90       _prefs_dialog_setup        0040fe90 f   prefs_dialog.obj
 0001:0000f4b0       _prefs_dialog_set_defaults 004104b0 f   prefs_dialog.obj
 0001:0000fc10       _prefs_dialog_ok           00410c10 f   prefs_dialog.obj
 0001:000104c0       _prefs_dialog_auth         004114c0 f   prefs_dialog_auth.obj
 0001:00010f30       _prefs_dialog_misc         00411f30 f   prefs_dialog_misc.obj
 0001:000110b0       _prefs_dialog_plugins_prefs 004120b0 f   prefs_dialog_plugins_prefs.obj
 0001:000111d0       _prefs_dialog_plugins_prefs_fill 004121d0 f   prefs_dialog_plugins_prefs.obj
 0001:000112f0       _prefs_plugins_reset       004122f0 f   prefs_dialog_plugins_prefs.obj
 0001:000114b0       _prefs_plugins_prefs_redraw 004124b0 f   prefs_dialog_plugins_prefs.obj
 0001:00011b70       _prefs_dialog_scan_opt     00412b70 f   prefs_dialog_scan_opt.obj
 0001:00011fa0       _fill_scanner_list         00412fa0 f   prefs_dialog_scan_opt.obj
 0001:00012250       _prefs_scanner_redraw      00413250 f   prefs_dialog_scan_opt.obj
 0001:00012300       _dialog_delete_key         00413300 f   prefs_dialog_user.obj
 0001:00012410       _prefs_dialog_user         00413410 f   prefs_dialog_user.obj
 0001:00012cc0       _prefs_dialog_plugins      00413cc0 f   prefs_plugins.obj
 0001:00013970       _prefs_plugins_redraw      00414970 f   prefs_plugins.obj
 0001:000139b0       _fill_plugins_family       004149b0 f   prefs_plugins.obj
 0001:00013ec0       _prefs_dialog_target_free_list 00414ec0 f   prefs_target.obj
 0001:00013f40       _prefs_dialog_target_fill_sessions 00414f40 f   prefs_target.obj
 0001:000140b0       _prefs_dialog_target       004150b0 f   prefs_target.obj
 0001:000142f0       _load_font_conversions     004152f0 f   gdc.obj
 0001:00014330       _cnt_nl                    00415330 f   gdc.obj
 0001:00014390       _GDCImageStringNL          00415390 f   gdc.obj
 0001:00014450       _GDC_destroy_image         00415450 f   gdc.obj
 0001:00014460       _out_err                   00415460 f   gdc.obj
 0001:00014550       _price_to_str              00415550 f   price_conv.obj
 0001:00014780       _pie_gif                   00415780 f   gdc_pie.obj
 0001:00017a80       _draw_3d_line              00418a80 f   gdchart.obj
 0001:00017d40       _draw_3d_area              00418d40 f   gdchart.obj
 0001:000180e0       _draw_3d_bar               004190e0 f   gdchart.obj
 0001:00018220       _out_graph                 00419220 f   gdchart.obj
 0001:0001d8f0       _gdImageCreate             0041e8f0 f   gd.obj
 0001:0001d980       _gdImageDestroy            0041e980 f   gd.obj
 0001:0001d9e0       _gdImageColorClosest       0041e9e0 f   gd.obj
 0001:0001da80       _gdImageColorExact         0041ea80 f   gd.obj
 0001:0001dad0       _gdImageColorAllocate      0041ead0 f   gd.obj
 0001:0001db40       _gdImageColorDeallocate    0041eb40 f   gd.obj
 0001:0001db60       _gdImageColorTransparent   0041eb60 f   gd.obj
 0001:0001db70       _gdImageSetPixel           0041eb70 f   gd.obj
 0001:0001ddc0       _gdImageGetPixel           0041edc0 f   gd.obj
 0001:0001de00       _gdImageLine               0041ee00 f   gd.obj
 0001:0001dfe0       _gdImageDashedLine         0041efe0 f   gd.obj
 0001:0001e270       _gdImageBoundsSafe         0041f270 f   gd.obj
 0001:0001e2a0       _gdImageChar               0041f2a0 f   gd.obj
 0001:0001e350       _gdImageCharUp             0041f350 f   gd.obj
 0001:0001e410       _gdImageString             0041f410 f   gd.obj
 0001:0001e470       _gdImageStringUp           0041f470 f   gd.obj
 0001:0001e4d0       _gdImageString16           0041f4d0 f   gd.obj
 0001:0001e520       _gdImageStringUp16         0041f520 f   gd.obj
 0001:0001e590       _gdImageArc                0041f590 f   gd.obj
 0001:0001e6a0       _gdImageFillToBorder       0041f6a0 f   gd.obj
 0001:0001e810       _gdImageFill               0041f810 f   gd.obj
 0001:0001e9d0       _gdImageGif                0041f9d0 f   gd.obj
 0001:0001f430       _gdImageCreateFromGif      00420430 f   gd.obj
 0001:0001ffa0       _gdImageRectangle          00420fa0 f   gd.obj
 0001:00020010       _gdImageFilledRectangle    00421010 f   gd.obj
 0001:00020060       _gdImageCopy               00421060 f   gd.obj
 0001:000201f0       _gdImageCopyResized        004211f0 f   gd.obj
 0001:00020550       _gdGetWord                 00421550 f   gd.obj
 0001:000205a0       _gdPutWord                 004215a0 f   gd.obj
 0001:000205d0       _gdGetByte                 004215d0 f   gd.obj
 0001:00020600       _gdImageCreateFromGd       00421600 f   gd.obj
 0001:00020730       _gdImageGd                 00421730 f   gd.obj
 0001:00020810       _gdImageCreateFromXbm      00421810 f   gd.obj
 0001:00020a50       _gdImagePolygon            00421a50 f   gd.obj
 0001:00020ac0       _gdImageFilledPolygon      00421ac0 f   gd.obj
 0001:00020d50       _gdCompareInt              00421d50 f   gd.obj
 0001:00020d60       _gdImageSetStyle           00421d60 f   gd.obj
 0001:00020dd0       _gdImageSetBrush           00421dd0 f   gd.obj
 0001:00020e70       _gdImageSetTile            00421e70 f   gd.obj
 0001:00020f10       _gdImageInterlace          00421f10 f   gd.obj
 0001:00020f20       _harg_add                  00421f20 f   nessus:nessus.dll
 0001:00020f26       _harg_create               00421f26 f   nessus:nessus.dll
 0001:00020f2c       _harg_get_tvalue           00421f2c f   nessus:nessus.dll
 0001:00020f32       _get_optind                00421f32 f   nessus:nessus.dll
 0001:00020f38       _inc_optind                00421f38 f   nessus:nessus.dll
 0001:00020f3e       _get_optarg                00421f3e f   nessus:nessus.dll
 0001:00020f44       _getopt_long               00421f44 f   nessus:nessus.dll
 0001:00020f4a       _harg_close                00421f4a f   nessus:nessus.dll
 0001:00020f50       _harg_walk_next            00421f50 f   nessus:nessus.dll
 0001:00020f56       _harg_walk_init            00421f56 f   nessus:nessus.dll
 0001:00020f5c       _io_send                   00421f5c f   peks:peks.dll
 0001:00020f62       _io_recv                   00421f62 f   peks:peks.dll
 0001:00020f68       _io_ctrl                   00421f68 f   peks:peks.dll
 0001:00020f6e       ___peks_nt_fprintf         00421f6e f   peks:peks.dll
 0001:00020f74       _peks_strerr               00421f74 f   peks:peks.dll
 0001:00020f7a       _io_thtrp                  00421f7a f   peks:peks.dll
 0001:00020f80       _io_shutdown               00421f80 f   peks:peks.dll
 0001:00020f86       _peks_client_authenticate  00421f86 f   peks:peks.dll
 0001:00020f8c       _client_negotiate_session_key 00421f8c f   peks:peks.dll
 0001:00020f92       ___peks_nt_printf          00421f92 f   peks:peks.dll
 0001:00020f98       ___peks_nt_setconsole      00421f98 f   peks:peks.dll
 0001:00020f9e       _peks_set_keep_alive_notice 00421f9e f   peks:peks.dll
 0001:00020fa4       _peks_set_uservar          00421fa4 f   peks:peks.dll
 0001:00020faa       _peks_set_homevar          00421faa f   peks:peks.dll
 0001:00020fb0       _peks_version              00421fb0 f   peks:peks.dll
 0001:00020fb6       ___peks_nt_exit            00421fb6 f   peks:peks.dll
 0001:00020fbc       _peks_save_public_key      00421fbc f   peks:peks.dll
 0001:00020fc2       _peks_get_username         00421fc2 f   peks:peks.dll
 0001:00020fc8       _peks_list_keyfile         00421fc8 f   peks:peks.dll
 0001:00020fce       _peks_delete_hostkey       00421fce f   peks:peks.dll
 0001:00020fd4       _peks_delete_userkey       00421fd4 f   peks:peks.dll
 0001:00020fda       _peks_save_private_key     00421fda f   peks:peks.dll
 0001:00020fe0       _peks_private_key          00421fe0 f   peks:peks.dll
 0001:00020fe6       ___peks_nt_getpass         00421fe6 f   peks:peks.dll
 0001:00020fec       _pmalloc                   00421fec f   peks:peks.dll
 0001:00020ff2       _peks_get_homedir          00421ff2 f   peks:peks.dll
 0001:00020ff8       _xfree                     00421ff8 f   peks:peks.dll
 0001:00020ffe       _peks_get_dirfile          00421ffe f   peks:peks.dll
 0001:00021004       ___peks_nt_fgets           00422004 f   peks:peks.dll
 0001:0002100a       ___peks_nt_fopen           0042200a f   peks:peks.dll
 0001:00021010       ___peks_nt_read            00422010 f   peks:peks.dll
 0001:00021016       ___peks_nt_open            00422016 f   peks:peks.dll
 0001:0002101c       _io_close                  0042201c f   peks:peks.dll
 0001:00021022       ___peks_nt_close           00422022 f   peks:peks.dll
 0001:00021028       _find_classes_by_name      00422028 f   peks:peks.dll
 0001:0002102e       _gtk_pixmap_new            0042202e f   gtk-1.3:gtk-1.3.dll
 0001:00021034       _gtk_widget_get_style      00422034 f   gtk-1.3:gtk-1.3.dll
 0001:0002103a       _gtk_widget_realize        0042203a f   gtk-1.3:gtk-1.3.dll
 0001:00021040       _gtk_widget_grab_default   00422040 f   gtk-1.3:gtk-1.3.dll
 0001:00021046       _gtk_table_attach_defaults 00422046 f   gtk-1.3:gtk-1.3.dll
 0001:0002104c       _gtk_table_get_type        0042204c f   gtk-1.3:gtk-1.3.dll
 0001:00021052       _gtk_table_new             00422052 f   gtk-1.3:gtk-1.3.dll
 0001:00021058       _gtk_button_new_with_label 00422058 f   gtk-1.3:gtk-1.3.dll
 0001:0002105e       _gtk_box_pack_end          0042205e f   gtk-1.3:gtk-1.3.dll
 0001:00021064       _gtk_label_set_justify     00422064 f   gtk-1.3:gtk-1.3.dll
 0001:0002106a       _gtk_label_get_type        0042206a f   gtk-1.3:gtk-1.3.dll
 0001:00021070       _gtk_label_new             00422070 f   gtk-1.3:gtk-1.3.dll
 0001:00021076       _gtk_box_pack_start        00422076 f   gtk-1.3:gtk-1.3.dll
 0001:0002107c       _gtk_box_get_type          0042207c f   gtk-1.3:gtk-1.3.dll
 0001:00021082       _gtk_hbox_new              00422082 f   gtk-1.3:gtk-1.3.dll
 0001:00021088       _gtk_widget_show           00422088 f   gtk-1.3:gtk-1.3.dll
 0001:0002108e       _gtk_container_add         0042208e f   gtk-1.3:gtk-1.3.dll
 0001:00021094       _gtk_container_set_border_width 00422094 f   gtk-1.3:gtk-1.3.dll
 0001:0002109a       _gtk_container_get_type    0042209a f   gtk-1.3:gtk-1.3.dll
 0001:000210a0       _gtk_vbox_new              004220a0 f   gtk-1.3:gtk-1.3.dll
 0001:000210a6       _gtk_window_set_position   004220a6 f   gtk-1.3:gtk-1.3.dll
 0001:000210ac       _gtk_signal_connect        004220ac f   gtk-1.3:gtk-1.3.dll
 0001:000210b2       _gtk_window_set_title      004220b2 f   gtk-1.3:gtk-1.3.dll
 0001:000210b8       _gtk_type_check_object_cast 004220b8 f   gtk-1.3:gtk-1.3.dll
 0001:000210be       _gtk_window_get_type       004220be f   gtk-1.3:gtk-1.3.dll
 0001:000210c4       _gtk_window_new            004220c4 f   gtk-1.3:gtk-1.3.dll
 0001:000210ca       _gtk_grab_add              004220ca f   gtk-1.3:gtk-1.3.dll
 0001:000210d0       _gtk_grab_remove           004220d0 f   gtk-1.3:gtk-1.3.dll
 0001:000210d6       _gtk_main_iteration        004220d6 f   gtk-1.3:gtk-1.3.dll
 0001:000210dc       _gtk_events_pending        004220dc f   gtk-1.3:gtk-1.3.dll
 0001:000210e2       _gtk_idle_add              004220e2 f   gtk-1.3:gtk-1.3.dll
 0001:000210e8       _gtk_scrolled_window_add_with_viewport 004220e8 f   gtk-1.3:gtk-1.3.dll
 0001:000210ee       _gtk_list_new              004220ee f   gtk-1.3:gtk-1.3.dll
 0001:000210f4       _gtk_scrolled_window_set_policy 004220f4 f   gtk-1.3:gtk-1.3.dll
 0001:000210fa       _gtk_scrolled_window_get_type 004220fa f   gtk-1.3:gtk-1.3.dll
 0001:00021100       _gtk_scrolled_window_new   00422100 f   gtk-1.3:gtk-1.3.dll
 0001:00021106       _gtk_window_set_default_size 00422106 f   gtk-1.3:gtk-1.3.dll
 0001:0002110c       _gtk_object_set_data       0042210c f   gtk-1.3:gtk-1.3.dll
 0001:00021112       _gtk_list_remove_items     00422112 f   gtk-1.3:gtk-1.3.dll
 0001:00021118       _gtk_list_get_type         00422118 f   gtk-1.3:gtk-1.3.dll
 0001:0002111e       _gtk_object_get_data       0042211e f   gtk-1.3:gtk-1.3.dll
 0001:00021124       _gtk_idle_remove           00422124 f   gtk-1.3:gtk-1.3.dll
 0001:0002112a       _gtk_widget_hide           0042212a f   gtk-1.3:gtk-1.3.dll
 0001:00021130       _gtk_widget_destroy        00422130 f   gtk-1.3:gtk-1.3.dll
 0001:00021136       _gtk_progress_bar_update   00422136 f   gtk-1.3:gtk-1.3.dll
 0001:0002113c       _gtk_progress_bar_get_type 0042213c f   gtk-1.3:gtk-1.3.dll
 0001:00021142       _gtk_label_set_text        00422142 f   gtk-1.3:gtk-1.3.dll
 0001:00021148       _gtk_list_append_items     00422148 f   gtk-1.3:gtk-1.3.dll
 0001:0002114e       _gtk_hseparator_new        0042214e f   gtk-1.3:gtk-1.3.dll
 0001:00021154       _gtk_progress_bar_new      00422154 f   gtk-1.3:gtk-1.3.dll
 0001:0002115a       _gtk_widget_set_usize      0042215a f   gtk-1.3:gtk-1.3.dll
 0001:00021160       _gtk_table_set_row_spacings 00422160 f   gtk-1.3:gtk-1.3.dll
 0001:00021166       _gtk_table_set_col_spacings 00422166 f   gtk-1.3:gtk-1.3.dll
 0001:0002116c       _gtk_list_item_new         0042216c f   gtk-1.3:gtk-1.3.dll
 0001:00021172       _gtk_main                  00422172 f   gtk-1.3:gtk-1.3.dll
 0001:00021178       _gtk_entry_set_visibility  00422178 f   gtk-1.3:gtk-1.3.dll
 0001:0002117e       _gtk_entry_get_type        0042217e f   gtk-1.3:gtk-1.3.dll
 0001:00021184       _gtk_entry_new             00422184 f   gtk-1.3:gtk-1.3.dll
 0001:0002118a       _gtk_vseparator_new        0042218a f   gtk-1.3:gtk-1.3.dll
 0001:00021190       _gtk_entry_get_text        00422190 f   gtk-1.3:gtk-1.3.dll
 0001:00021196       _gtk_text_insert           00422196 f   gtk-1.3:gtk-1.3.dll
 0001:0002119c       _gtk_text_set_word_wrap    0042219c f   gtk-1.3:gtk-1.3.dll
 0001:000211a2       _gtk_text_set_editable     004221a2 f   gtk-1.3:gtk-1.3.dll
 0001:000211a8       _gtk_text_get_type         004221a8 f   gtk-1.3:gtk-1.3.dll
 0001:000211ae       _gtk_table_attach          004221ae f   gtk-1.3:gtk-1.3.dll
 0001:000211b4       _gtk_text_new              004221b4 f   gtk-1.3:gtk-1.3.dll
 0001:000211ba       _gtk_vscrollbar_new        004221ba f   gtk-1.3:gtk-1.3.dll
 0001:000211c0       _gtk_adjustment_new        004221c0 f   gtk-1.3:gtk-1.3.dll
 0001:000211c6       _gtk_adjustment_get_type   004221c6 f   gtk-1.3:gtk-1.3.dll
 0001:000211cc       _gtk_file_selection_set_filename 004221cc f   gtk-1.3:gtk-1.3.dll
 0001:000211d2       _gtk_file_selection_get_type 004221d2 f   gtk-1.3:gtk-1.3.dll
 0001:000211d8       _gtk_file_selection_new    004221d8 f   gtk-1.3:gtk-1.3.dll
 0001:000211de       _gtk_file_selection_get_filename 004221de f   gtk-1.3:gtk-1.3.dll
 0001:000211e4       _gtk_entry_set_text        004221e4 f   gtk-1.3:gtk-1.3.dll
 0001:000211ea       _gtk_tree_item_collapse    004221ea f   gtk-1.3:gtk-1.3.dll
 0001:000211f0       _gtk_tree_item_expand      004221f0 f   gtk-1.3:gtk-1.3.dll
 0001:000211f6       _gtk_tree_item_set_subtree 004221f6 f   gtk-1.3:gtk-1.3.dll
 0001:000211fc       _gtk_tree_item_get_type    004221fc f   gtk-1.3:gtk-1.3.dll
 0001:00021202       _gtk_tree_append           00422202 f   gtk-1.3:gtk-1.3.dll
 0001:00021208       _gtk_tree_get_type         00422208 f   gtk-1.3:gtk-1.3.dll
 0001:0002120e       _gtk_tree_item_new         0042220e f   gtk-1.3:gtk-1.3.dll
 0001:00021214       _gtk_tree_new              00422214 f   gtk-1.3:gtk-1.3.dll
 0001:0002121a       _gtk_option_menu_set_history 0042221a f   gtk-1.3:gtk-1.3.dll
 0001:00021220       _gtk_menu_append           00422220 f   gtk-1.3:gtk-1.3.dll
 0001:00021226       _gtk_menu_get_type         00422226 f   gtk-1.3:gtk-1.3.dll
 0001:0002122c       _gtk_menu_item_new_with_label 0042222c f   gtk-1.3:gtk-1.3.dll
 0001:00021232       _gtk_option_menu_set_menu  00422232 f   gtk-1.3:gtk-1.3.dll
 0001:00021238       _gtk_option_menu_get_type  00422238 f   gtk-1.3:gtk-1.3.dll
 0001:0002123e       _gtk_menu_new              0042223e f   gtk-1.3:gtk-1.3.dll
 0001:00021244       _gtk_option_menu_new       00422244 f   gtk-1.3:gtk-1.3.dll
 0001:0002124a       _gtk_paned_add2            0042224a f   gtk-1.3:gtk-1.3.dll
 0001:00021250       _gtk_paned_add1            00422250 f   gtk-1.3:gtk-1.3.dll
 0001:00021256       _gtk_paned_get_type        00422256 f   gtk-1.3:gtk-1.3.dll
 0001:0002125c       _gtk_hpaned_new            0042225c f   gtk-1.3:gtk-1.3.dll
 0001:00021262       _gtk_widget_map            00422262 f   gtk-1.3:gtk-1.3.dll
 0001:00021268       _gtk_adjustment_set_value  00422268 f   gtk-1.3:gtk-1.3.dll
 0001:0002126e       _gtk_scrolled_window_get_vadjustment 0042226e f   gtk-1.3:gtk-1.3.dll
 0001:00021274       _gtk_menu_get_active       00422274 f   gtk-1.3:gtk-1.3.dll
 0001:0002127a       _gtk_init                  0042227a f   gtk-1.3:gtk-1.3.dll
 0001:00021280       _gtk_main_quit             00422280 f   gtk-1.3:gtk-1.3.dll
 0001:00021286       _gtk_frame_new             00422286 f   gtk-1.3:gtk-1.3.dll
 0001:0002128c       _gtk_notebook_append_page  0042228c f   gtk-1.3:gtk-1.3.dll
 0001:00021292       _gtk_notebook_set_tab_pos  00422292 f   gtk-1.3:gtk-1.3.dll
 0001:00021298       _gtk_notebook_get_type     00422298 f   gtk-1.3:gtk-1.3.dll
 0001:0002129e       _gtk_notebook_new          0042229e f   gtk-1.3:gtk-1.3.dll
 0001:000212a4       _gtk_toggle_button_set_active 004222a4 f   gtk-1.3:gtk-1.3.dll
 0001:000212aa       _gtk_toggle_button_get_type 004222aa f   gtk-1.3:gtk-1.3.dll
 0001:000212b0       _gtk_tooltips_enable       004222b0 f   gtk-1.3:gtk-1.3.dll
 0001:000212b6       _gtk_tooltips_set_tip      004222b6 f   gtk-1.3:gtk-1.3.dll
 0001:000212bc       _gtk_tooltips_new          004222bc f   gtk-1.3:gtk-1.3.dll
 0001:000212c2       _gtk_notebook_set_page     004222c2 f   gtk-1.3:gtk-1.3.dll
 0001:000212c8       _gtk_check_button_new_with_label 004222c8 f   gtk-1.3:gtk-1.3.dll
 0001:000212ce       _gtk_container_remove      004222ce f   gtk-1.3:gtk-1.3.dll
 0001:000212d4       _gtk_radio_button_group    004222d4 f   gtk-1.3:gtk-1.3.dll
 0001:000212da       _gtk_radio_button_get_type 004222da f   gtk-1.3:gtk-1.3.dll
 0001:000212e0       _gtk_radio_button_new_with_label 004222e0 f   gtk-1.3:gtk-1.3.dll
 0001:000212e6       _gtk_table_set_row_spacing 004222e6 f   gtk-1.3:gtk-1.3.dll
 0001:000212ec       _gtk_check_button_new      004222ec f   gtk-1.3:gtk-1.3.dll
 0001:000212f2       _gtk_table_set_col_spacing 004222f2 f   gtk-1.3:gtk-1.3.dll
 0001:000212f8       _gtk_object_remove_data    004222f8 f   gtk-1.3:gtk-1.3.dll
 0001:000212fe       _gtk_button_set_relief     004222fe f   gtk-1.3:gtk-1.3.dll
 0001:00021304       _gtk_button_get_type       00422304 f   gtk-1.3:gtk-1.3.dll
 0001:0002130a       _gtk_button_new            0042230a f   gtk-1.3:gtk-1.3.dll
 0001:00021310       _gtk_clist_remove          00422310 f   gtk-1.3:gtk-1.3.dll
 0001:00021316       _gtk_clist_append          00422316 f   gtk-1.3:gtk-1.3.dll
 0001:0002131c       _gtk_clist_get_type        0042231c f   gtk-1.3:gtk-1.3.dll
 0001:00021322       _gtk_clist_thaw            00422322 f   gtk-1.3:gtk-1.3.dll
 0001:00021328       _gtk_clist_set_column_width 00422328 f   gtk-1.3:gtk-1.3.dll
 0001:0002132e       _gtk_clist_optimal_column_width 0042232e f   gtk-1.3:gtk-1.3.dll
 0001:00021334       _gtk_clist_sort            00422334 f   gtk-1.3:gtk-1.3.dll
 0001:0002133a       _gtk_clist_set_row_data    0042233a f   gtk-1.3:gtk-1.3.dll
 0001:00021340       _gtk_clist_freeze          00422340 f   gtk-1.3:gtk-1.3.dll
 0001:00021346       _gdk_pixmap_create_from_xpm_d 00422346 f   gdk-1.3:gdk-1.3.dll
 0001:0002134c       _gdk_string_width          0042234c f   gdk-1.3:gdk-1.3.dll
 0001:00021352       _g_list_free               00422352 f   glib-1.3:glib-1.3.dll
 0001:00021358       _g_list_append             00422358 f   glib-1.3:glib-1.3.dll
 0001:0002135e       ___WSAFDIsSet@8            0042235e f   wsock32:WSOCK32.dll
 0001:00021364       _select@20                 00422364 f   wsock32:WSOCK32.dll
 0001:0002136a       _WSACleanup@0              0042236a f   wsock32:WSOCK32.dll
 0001:00021370       _WSAStartup@8              00422370 f   wsock32:WSOCK32.dll
 0001:00021380       __chkstk                   00422380 f   MSVCRT:chkstk.obj
 0001:00021380       __alloca_probe             00422380 f   MSVCRT:chkstk.obj
 0001:000213b0       __ftol                     004223b0 f   MSVCRT:MSVCRT.dll
 0001:000213b6       __CIpow                    004223b6 f   MSVCRT:MSVCRT.dll
 0001:000213bc       _WinMainCRTStartup         004223bc f   MSVCRT:crtexew.obj
 0001:0002151a       __XcptFilter               0042251a f   MSVCRT:MSVCRT.dll
 0001:00021520       __initterm                 00422520 f   MSVCRT:MSVCRT.dll
 0001:00021526       __setdefaultprecision      00422526 f   MSVCRT:fp8.obj
 0001:00021538       __matherr                  00422538 f   MSVCRT:merr.obj
 0001:0002153b       __setargv                  0042253b f   MSVCRT:dllargv.obj
 0001:0002153c       __except_handler3          0042253c f   MSVCRT:MSVCRT.dll
 0001:00021542       __controlfp                00422542 f   MSVCRT:MSVCRT.dll
 0001:00021550       _chdir                     00422550 f   MSVCRT:MSVCRT.dll
 0001:00021550       __chdir                    00422550 f   MSVCRT:MSVCRT.dll
 0001:00021556       _mkdir                     00422556 f   MSVCRT:MSVCRT.dll
 0001:00021556       __mkdir                    00422556 f   MSVCRT:MSVCRT.dll
 0002:00000000       __imp__GetStartupInfoA@4   00423000     kernel32:KERNEL32.dll
 0002:00000004       __imp__GetModuleHandleA@4  00423004     kernel32:KERNEL32.dll
 0002:00000008       \177KERNEL32_NULL_THUNK_DATA 00423008     kernel32:KERNEL32.dll
 0002:0000000c       __imp__strdup              0042300c     MSVCRT:MSVCRT.dll
 0002:0000000c       __imp___strdup             0042300c     MSVCRT:MSVCRT.dll
 0002:00000010       __imp___chdir              00423010     MSVCRT:MSVCRT.dll
 0002:00000014       __imp___mkdir              00423014     MSVCRT:MSVCRT.dll
 0002:00000018       __imp__fflush              00423018     MSVCRT:MSVCRT.dll
 0002:0000001c       __imp___controlfp          0042301c     MSVCRT:MSVCRT.dll
 0002:00000020       __imp___except_handler3    00423020     MSVCRT:MSVCRT.dll
 0002:00000024       __imp____set_app_type      00423024     MSVCRT:MSVCRT.dll
 0002:00000028       __imp____p__fmode          00423028     MSVCRT:MSVCRT.dll
 0002:0000002c       __imp____p__commode        0042302c     MSVCRT:MSVCRT.dll
 0002:00000030       __imp___adjust_fdiv        00423030     MSVCRT:MSVCRT.dll
 0002:00000034       __imp____setusermatherr    00423034     MSVCRT:MSVCRT.dll
 0002:00000038       __imp___initterm           00423038     MSVCRT:MSVCRT.dll
 0002:0000003c       __imp____getmainargs       0042303c     MSVCRT:MSVCRT.dll
 0002:00000040       __imp___acmdln             00423040     MSVCRT:MSVCRT.dll
 0002:00000044       __imp___XcptFilter         00423044     MSVCRT:MSVCRT.dll
 0002:00000048       __imp__realloc             00423048     MSVCRT:MSVCRT.dll
 0002:0000004c       __imp__putc                0042304c     MSVCRT:MSVCRT.dll
 0002:00000050       __imp__getc                00423050     MSVCRT:MSVCRT.dll
 0002:00000054       __imp__fread               00423054     MSVCRT:MSVCRT.dll
 0002:00000058       __imp__fwrite              00423058     MSVCRT:MSVCRT.dll
 0002:0000005c       __imp__fputc               0042305c     MSVCRT:MSVCRT.dll
 0002:00000060       __imp__calloc              00423060     MSVCRT:MSVCRT.dll
 0002:00000064       __imp__strcspn             00423064     MSVCRT:MSVCRT.dll
 0002:00000068       __imp__atof                00423068     MSVCRT:MSVCRT.dll
 0002:0000006c       __imp__ceil                0042306c     MSVCRT:MSVCRT.dll
 0002:00000070       __imp__floor               00423070     MSVCRT:MSVCRT.dll
 0002:00000074       __imp__qsort               00423074     MSVCRT:MSVCRT.dll
 0002:00000078       __imp___CIpow              00423078     MSVCRT:MSVCRT.dll
 0002:0000007c       __imp__perror              0042307c     MSVCRT:MSVCRT.dll
 0002:00000080       __imp__strncat             00423080     MSVCRT:MSVCRT.dll
 0002:00000084       __imp__exit                00423084     MSVCRT:MSVCRT.dll
 0002:00000088       __imp__strtok              00423088     MSVCRT:MSVCRT.dll
 0002:0000008c       __imp___strnicmp           0042308c     MSVCRT:MSVCRT.dll
 0002:00000090       __imp___ftol               00423090     MSVCRT:MSVCRT.dll
 0002:00000094       __imp__memmove             00423094     MSVCRT:MSVCRT.dll
 0002:00000098       __imp__fgets               00423098     MSVCRT:MSVCRT.dll
 0002:0000009c       __imp__fopen               0042309c     MSVCRT:MSVCRT.dll
 0002:000000a0       __imp__fprintf             004230a0     MSVCRT:MSVCRT.dll
 0002:000000a4       __imp___isctype            004230a4     MSVCRT:MSVCRT.dll
 0002:000000a8       __imp____mb_cur_max        004230a8     MSVCRT:MSVCRT.dll
 0002:000000ac       __imp___pctype             004230ac     MSVCRT:MSVCRT.dll
 0002:000000b0       __imp___exit               004230b0     MSVCRT:MSVCRT.dll
 0002:000000b4       __imp___stat               004230b4     MSVCRT:MSVCRT.dll
 0002:000000b8       __imp__strerror            004230b8     MSVCRT:MSVCRT.dll
 0002:000000bc       __imp__fclose              004230bc     MSVCRT:MSVCRT.dll
 0002:000000c0       __imp___putenv             004230c0     MSVCRT:MSVCRT.dll
 0002:000000c4       __imp__getenv              004230c4     MSVCRT:MSVCRT.dll
 0002:000000c8       __imp____p___argv          004230c8     MSVCRT:MSVCRT.dll
 0002:000000cc       __imp____p___argc          004230cc     MSVCRT:MSVCRT.dll
 0002:000000d0       __imp__malloc              004230d0     MSVCRT:MSVCRT.dll
 0002:000000d4       __imp__strrchr             004230d4     MSVCRT:MSVCRT.dll
 0002:000000d8       __imp___stricmp            004230d8     MSVCRT:MSVCRT.dll
 0002:000000dc       __imp__atoi                004230dc     MSVCRT:MSVCRT.dll
 0002:000000e0       __imp__free                004230e0     MSVCRT:MSVCRT.dll
 0002:000000e4       __imp__sscanf              004230e4     MSVCRT:MSVCRT.dll
 0002:000000e8       __imp__strstr              004230e8     MSVCRT:MSVCRT.dll
 0002:000000ec       __imp__strchr              004230ec     MSVCRT:MSVCRT.dll
 0002:000000f0       __imp__strncpy             004230f0     MSVCRT:MSVCRT.dll
 0002:000000f4       __imp___iob                004230f4     MSVCRT:MSVCRT.dll
 0002:000000f8       __imp___errno              004230f8     MSVCRT:MSVCRT.dll
 0002:000000fc       __imp__vsprintf            004230fc     MSVCRT:MSVCRT.dll
 0002:00000100       __imp__strncmp             00423100     MSVCRT:MSVCRT.dll
 0002:00000104       __imp__sprintf             00423104     MSVCRT:MSVCRT.dll
 0002:00000108       \177MSVCRT_NULL_THUNK_DATA 00423108     MSVCRT:MSVCRT.dll
 0002:0000010c       __imp____WSAFDIsSet@8      0042310c     wsock32:WSOCK32.dll
 0002:00000110       __imp__WSAStartup@8        00423110     wsock32:WSOCK32.dll
 0002:00000114       __imp__WSACleanup@0        00423114     wsock32:WSOCK32.dll
 0002:00000118       __imp__select@20           00423118     wsock32:WSOCK32.dll
 0002:0000011c       \177WSOCK32_NULL_THUNK_DATA 0042311c     wsock32:WSOCK32.dll
 0002:00000120       __imp__gdk_pixmap_create_from_xpm_d 00423120     gdk-1.3:gdk-1.3.dll
 0002:00000124       __imp__gdk_string_width    00423124     gdk-1.3:gdk-1.3.dll
 0002:00000128       \177gdk-1.3_NULL_THUNK_DATA 00423128     gdk-1.3:gdk-1.3.dll
 0002:0000012c       __imp__g_list_append       0042312c     glib-1.3:glib-1.3.dll
 0002:00000130       __imp__g_list_free         00423130     glib-1.3:glib-1.3.dll
 0002:00000134       \177glib-1.3_NULL_THUNK_DATA 00423134     glib-1.3:glib-1.3.dll
 0002:00000138       __imp__gtk_label_set_justify 00423138     gtk-1.3:gtk-1.3.dll
 0002:0000013c       __imp__gtk_label_get_type  0042313c     gtk-1.3:gtk-1.3.dll
 0002:00000140       __imp__gtk_label_new       00423140     gtk-1.3:gtk-1.3.dll
 0002:00000144       __imp__gtk_box_pack_end    00423144     gtk-1.3:gtk-1.3.dll
 0002:00000148       __imp__gtk_button_new_with_label 00423148     gtk-1.3:gtk-1.3.dll
 0002:0000014c       __imp__gtk_box_pack_start  0042314c     gtk-1.3:gtk-1.3.dll
 0002:00000150       __imp__gtk_hbox_new        00423150     gtk-1.3:gtk-1.3.dll
 0002:00000154       __imp__gtk_widget_show     00423154     gtk-1.3:gtk-1.3.dll
 0002:00000158       __imp__gtk_container_add   00423158     gtk-1.3:gtk-1.3.dll
 0002:0000015c       __imp__gtk_container_set_border_width 0042315c     gtk-1.3:gtk-1.3.dll
 0002:00000160       __imp__gtk_container_get_type 00423160     gtk-1.3:gtk-1.3.dll
 0002:00000164       __imp__gtk_box_get_type    00423164     gtk-1.3:gtk-1.3.dll
 0002:00000168       __imp__gtk_window_set_position 00423168     gtk-1.3:gtk-1.3.dll
 0002:0000016c       __imp__gtk_vbox_new        0042316c     gtk-1.3:gtk-1.3.dll
 0002:00000170       __imp__gtk_window_set_title 00423170     gtk-1.3:gtk-1.3.dll
 0002:00000174       __imp__gtk_type_check_object_cast 00423174     gtk-1.3:gtk-1.3.dll
 0002:00000178       __imp__gtk_window_get_type 00423178     gtk-1.3:gtk-1.3.dll
 0002:0000017c       __imp__gtk_window_new      0042317c     gtk-1.3:gtk-1.3.dll
 0002:00000180       __imp__gtk_grab_add        00423180     gtk-1.3:gtk-1.3.dll
 0002:00000184       __imp__gtk_grab_remove     00423184     gtk-1.3:gtk-1.3.dll
 0002:00000188       __imp__gtk_main_iteration  00423188     gtk-1.3:gtk-1.3.dll
 0002:0000018c       __imp__gtk_events_pending  0042318c     gtk-1.3:gtk-1.3.dll
 0002:00000190       __imp__gtk_idle_add        00423190     gtk-1.3:gtk-1.3.dll
 0002:00000194       __imp__gtk_scrolled_window_add_with_viewport 00423194     gtk-1.3:gtk-1.3.dll
 0002:00000198       __imp__gtk_list_new        00423198     gtk-1.3:gtk-1.3.dll
 0002:0000019c       __imp__gtk_signal_connect  0042319c     gtk-1.3:gtk-1.3.dll
 0002:000001a0       __imp__gtk_table_get_type  004231a0     gtk-1.3:gtk-1.3.dll
 0002:000001a4       __imp__gtk_scrolled_window_new 004231a4     gtk-1.3:gtk-1.3.dll
 0002:000001a8       __imp__gtk_window_set_default_size 004231a8     gtk-1.3:gtk-1.3.dll
 0002:000001ac       __imp__gtk_object_set_data 004231ac     gtk-1.3:gtk-1.3.dll
 0002:000001b0       __imp__gtk_list_remove_items 004231b0     gtk-1.3:gtk-1.3.dll
 0002:000001b4       __imp__gtk_list_get_type   004231b4     gtk-1.3:gtk-1.3.dll
 0002:000001b8       __imp__gtk_object_get_data 004231b8     gtk-1.3:gtk-1.3.dll
 0002:000001bc       __imp__gtk_idle_remove     004231bc     gtk-1.3:gtk-1.3.dll
 0002:000001c0       __imp__gtk_widget_hide     004231c0     gtk-1.3:gtk-1.3.dll
 0002:000001c4       __imp__gtk_widget_destroy  004231c4     gtk-1.3:gtk-1.3.dll
 0002:000001c8       __imp__gtk_progress_bar_update 004231c8     gtk-1.3:gtk-1.3.dll
 0002:000001cc       __imp__gtk_progress_bar_get_type 004231cc     gtk-1.3:gtk-1.3.dll
 0002:000001d0       __imp__gtk_label_set_text  004231d0     gtk-1.3:gtk-1.3.dll
 0002:000001d4       __imp__gtk_list_append_items 004231d4     gtk-1.3:gtk-1.3.dll
 0002:000001d8       __imp__gtk_hseparator_new  004231d8     gtk-1.3:gtk-1.3.dll
 0002:000001dc       __imp__gtk_progress_bar_new 004231dc     gtk-1.3:gtk-1.3.dll
 0002:000001e0       __imp__gtk_widget_set_usize 004231e0     gtk-1.3:gtk-1.3.dll
 0002:000001e4       __imp__gtk_table_set_row_spacings 004231e4     gtk-1.3:gtk-1.3.dll
 0002:000001e8       __imp__gtk_table_set_col_spacings 004231e8     gtk-1.3:gtk-1.3.dll
 0002:000001ec       __imp__gtk_list_item_new   004231ec     gtk-1.3:gtk-1.3.dll
 0002:000001f0       __imp__gtk_main            004231f0     gtk-1.3:gtk-1.3.dll
 0002:000001f4       __imp__gtk_entry_set_visibility 004231f4     gtk-1.3:gtk-1.3.dll
 0002:000001f8       __imp__gtk_entry_get_type  004231f8     gtk-1.3:gtk-1.3.dll
 0002:000001fc       __imp__gtk_entry_new       004231fc     gtk-1.3:gtk-1.3.dll
 0002:00000200       __imp__gtk_vseparator_new  00423200     gtk-1.3:gtk-1.3.dll
 0002:00000204       __imp__gtk_entry_get_text  00423204     gtk-1.3:gtk-1.3.dll
 0002:00000208       __imp__gtk_text_insert     00423208     gtk-1.3:gtk-1.3.dll
 0002:0000020c       __imp__gtk_text_set_word_wrap 0042320c     gtk-1.3:gtk-1.3.dll
 0002:00000210       __imp__gtk_text_set_editable 00423210     gtk-1.3:gtk-1.3.dll
 0002:00000214       __imp__gtk_text_get_type   00423214     gtk-1.3:gtk-1.3.dll
 0002:00000218       __imp__gtk_table_attach    00423218     gtk-1.3:gtk-1.3.dll
 0002:0000021c       __imp__gtk_text_new        0042321c     gtk-1.3:gtk-1.3.dll
 0002:00000220       __imp__gtk_vscrollbar_new  00423220     gtk-1.3:gtk-1.3.dll
 0002:00000224       __imp__gtk_adjustment_new  00423224     gtk-1.3:gtk-1.3.dll
 0002:00000228       __imp__gtk_file_selection_new 00423228     gtk-1.3:gtk-1.3.dll
 0002:0000022c       __imp__gtk_pixmap_new      0042322c     gtk-1.3:gtk-1.3.dll
 0002:00000230       __imp__gtk_table_attach_defaults 00423230     gtk-1.3:gtk-1.3.dll
 0002:00000234       __imp__gtk_table_new       00423234     gtk-1.3:gtk-1.3.dll
 0002:00000238       __imp__gtk_file_selection_get_filename 00423238     gtk-1.3:gtk-1.3.dll
 0002:0000023c       __imp__gtk_entry_set_text  0042323c     gtk-1.3:gtk-1.3.dll
 0002:00000240       __imp__gtk_tree_item_collapse 00423240     gtk-1.3:gtk-1.3.dll
 0002:00000244       __imp__gtk_tree_item_expand 00423244     gtk-1.3:gtk-1.3.dll
 0002:00000248       __imp__gtk_tree_item_set_subtree 00423248     gtk-1.3:gtk-1.3.dll
 0002:0000024c       __imp__gtk_tree_item_get_type 0042324c     gtk-1.3:gtk-1.3.dll
 0002:00000250       __imp__gtk_tree_append     00423250     gtk-1.3:gtk-1.3.dll
 0002:00000254       __imp__gtk_tree_get_type   00423254     gtk-1.3:gtk-1.3.dll
 0002:00000258       __imp__gtk_tree_item_new   00423258     gtk-1.3:gtk-1.3.dll
 0002:0000025c       __imp__gtk_tree_new        0042325c     gtk-1.3:gtk-1.3.dll
 0002:00000260       __imp__gtk_option_menu_set_history 00423260     gtk-1.3:gtk-1.3.dll
 0002:00000264       __imp__gtk_menu_append     00423264     gtk-1.3:gtk-1.3.dll
 0002:00000268       __imp__gtk_menu_get_type   00423268     gtk-1.3:gtk-1.3.dll
 0002:0000026c       __imp__gtk_menu_item_new_with_label 0042326c     gtk-1.3:gtk-1.3.dll
 0002:00000270       __imp__gtk_option_menu_set_menu 00423270     gtk-1.3:gtk-1.3.dll
 0002:00000274       __imp__gtk_option_menu_get_type 00423274     gtk-1.3:gtk-1.3.dll
 0002:00000278       __imp__gtk_menu_new        00423278     gtk-1.3:gtk-1.3.dll
 0002:0000027c       __imp__gtk_option_menu_new 0042327c     gtk-1.3:gtk-1.3.dll
 0002:00000280       __imp__gtk_paned_add2      00423280     gtk-1.3:gtk-1.3.dll
 0002:00000284       __imp__gtk_paned_add1      00423284     gtk-1.3:gtk-1.3.dll
 0002:00000288       __imp__gtk_paned_get_type  00423288     gtk-1.3:gtk-1.3.dll
 0002:0000028c       __imp__gtk_hpaned_new      0042328c     gtk-1.3:gtk-1.3.dll
 0002:00000290       __imp__gtk_widget_map      00423290     gtk-1.3:gtk-1.3.dll
 0002:00000294       __imp__gtk_adjustment_set_value 00423294     gtk-1.3:gtk-1.3.dll
 0002:00000298       __imp__gtk_scrolled_window_get_vadjustment 00423298     gtk-1.3:gtk-1.3.dll
 0002:0000029c       __imp__gtk_menu_get_active 0042329c     gtk-1.3:gtk-1.3.dll
 0002:000002a0       __imp__gtk_init            004232a0     gtk-1.3:gtk-1.3.dll
 0002:000002a4       __imp__gtk_main_quit       004232a4     gtk-1.3:gtk-1.3.dll
 0002:000002a8       __imp__gtk_frame_new       004232a8     gtk-1.3:gtk-1.3.dll
 0002:000002ac       __imp__gtk_notebook_append_page 004232ac     gtk-1.3:gtk-1.3.dll
 0002:000002b0       __imp__gtk_notebook_set_tab_pos 004232b0     gtk-1.3:gtk-1.3.dll
 0002:000002b4       __imp__gtk_notebook_get_type 004232b4     gtk-1.3:gtk-1.3.dll
 0002:000002b8       __imp__gtk_notebook_new    004232b8     gtk-1.3:gtk-1.3.dll
 0002:000002bc       __imp__gtk_toggle_button_set_active 004232bc     gtk-1.3:gtk-1.3.dll
 0002:000002c0       __imp__gtk_toggle_button_get_type 004232c0     gtk-1.3:gtk-1.3.dll
 0002:000002c4       __imp__gtk_tooltips_enable 004232c4     gtk-1.3:gtk-1.3.dll
 0002:000002c8       __imp__gtk_tooltips_set_tip 004232c8     gtk-1.3:gtk-1.3.dll
 0002:000002cc       __imp__gtk_tooltips_new    004232cc     gtk-1.3:gtk-1.3.dll
 0002:000002d0       __imp__gtk_notebook_set_page 004232d0     gtk-1.3:gtk-1.3.dll
 0002:000002d4       __imp__gtk_check_button_new_with_label 004232d4     gtk-1.3:gtk-1.3.dll
 0002:000002d8       __imp__gtk_container_remove 004232d8     gtk-1.3:gtk-1.3.dll
 0002:000002dc       __imp__gtk_radio_button_group 004232dc     gtk-1.3:gtk-1.3.dll
 0002:000002e0       __imp__gtk_radio_button_get_type 004232e0     gtk-1.3:gtk-1.3.dll
 0002:000002e4       __imp__gtk_radio_button_new_with_label 004232e4     gtk-1.3:gtk-1.3.dll
 0002:000002e8       __imp__gtk_table_set_row_spacing 004232e8     gtk-1.3:gtk-1.3.dll
 0002:000002ec       __imp__gtk_check_button_new 004232ec     gtk-1.3:gtk-1.3.dll
 0002:000002f0       __imp__gtk_table_set_col_spacing 004232f0     gtk-1.3:gtk-1.3.dll
 0002:000002f4       __imp__gtk_object_remove_data 004232f4     gtk-1.3:gtk-1.3.dll
 0002:000002f8       __imp__gtk_button_set_relief 004232f8     gtk-1.3:gtk-1.3.dll
 0002:000002fc       __imp__gtk_button_get_type 004232fc     gtk-1.3:gtk-1.3.dll
 0002:00000300       __imp__gtk_button_new      00423300     gtk-1.3:gtk-1.3.dll
 0002:00000304       __imp__gtk_clist_remove    00423304     gtk-1.3:gtk-1.3.dll
 0002:00000308       __imp__gtk_clist_append    00423308     gtk-1.3:gtk-1.3.dll
 0002:0000030c       __imp__gtk_clist_get_type  0042330c     gtk-1.3:gtk-1.3.dll
 0002:00000310       __imp__gtk_clist_thaw      00423310     gtk-1.3:gtk-1.3.dll
 0002:00000314       __imp__gtk_clist_set_column_width 00423314     gtk-1.3:gtk-1.3.dll
 0002:00000318       __imp__gtk_clist_optimal_column_width 00423318     gtk-1.3:gtk-1.3.dll
 0002:0000031c       __imp__gtk_clist_sort      0042331c     gtk-1.3:gtk-1.3.dll
 0002:00000320       __imp__gtk_clist_set_row_data 00423320     gtk-1.3:gtk-1.3.dll
 0002:00000324       __imp__gtk_clist_freeze    00423324     gtk-1.3:gtk-1.3.dll
 0002:00000328       __imp__gtk_widget_grab_default 00423328     gtk-1.3:gtk-1.3.dll
 0002:0000032c       __imp__gtk_widget_realize  0042332c     gtk-1.3:gtk-1.3.dll
 0002:00000330       __imp__gtk_widget_get_style 00423330     gtk-1.3:gtk-1.3.dll
 0002:00000334       __imp__gtk_adjustment_get_type 00423334     gtk-1.3:gtk-1.3.dll
 0002:00000338       __imp__gtk_file_selection_set_filename 00423338     gtk-1.3:gtk-1.3.dll
 0002:0000033c       __imp__gtk_scrolled_window_set_policy 0042333c     gtk-1.3:gtk-1.3.dll
 0002:00000340       __imp__gtk_scrolled_window_get_type 00423340     gtk-1.3:gtk-1.3.dll
 0002:00000344       __imp__gtk_file_selection_get_type 00423344     gtk-1.3:gtk-1.3.dll
 0002:00000348       \177gtk-1.3_NULL_THUNK_DATA 00423348     gtk-1.3:gtk-1.3.dll
 0002:0000034c       __imp__arg_add_value       0042334c     nessus:nessus.dll
 0002:00000350       __imp__arg_set_value       00423350     nessus:nessus.dll
 0002:00000354       __imp__efree               00423354     nessus:nessus.dll
 0002:00000358       __imp__arg_get_value       00423358     nessus:nessus.dll
 0002:0000035c       __imp__emalloc             0042335c     nessus:nessus.dll
 0002:00000360       __imp__arg_set_type        00423360     nessus:nessus.dll
 0002:00000364       __imp__recv_line           00423364     nessus:nessus.dll
 0002:00000368       __imp__arg_get_type        00423368     nessus:nessus.dll
 0002:0000036c       __imp__plug_get_launch     0042336c     nessus:nessus.dll
 0002:00000370       __imp__plug_set_summary    00423370     nessus:nessus.dll
 0002:00000374       __imp__plug_set_description 00423374     nessus:nessus.dll
 0002:00000378       __imp__plug_set_family     00423378     nessus:nessus.dll
 0002:0000037c       __imp__plug_set_name       0042337c     nessus:nessus.dll
 0002:00000380       __imp__harg_add            00423380     nessus:nessus.dll
 0002:00000384       __imp__plug_set_copyright  00423384     nessus:nessus.dll
 0002:00000388       __imp__plug_get_family     00423388     nessus:nessus.dll
 0002:0000038c       __imp__plug_set_launch     0042338c     nessus:nessus.dll
 0002:00000390       __imp__harg_create         00423390     nessus:nessus.dll
 0002:00000394       __imp__estrdup             00423394     nessus:nessus.dll
 0002:00000398       __imp__arg_free            00423398     nessus:nessus.dll
 0002:0000039c       __imp__harg_get_tvalue     0042339c     nessus:nessus.dll
 0002:000003a0       __imp__open_sock_tcp_hn    004233a0     nessus:nessus.dll
 0002:000003a4       __imp__get_optind          004233a4     nessus:nessus.dll
 0002:000003a8       __imp__nn_resolve          004233a8     nessus:nessus.dll
 0002:000003ac       __imp__get_optarg          004233ac     nessus:nessus.dll
 0002:000003b0       __imp__getopt_long         004233b0     nessus:nessus.dll
 0002:000003b4       __imp__inc_optind          004233b4     nessus:nessus.dll
 0002:000003b8       __imp__append_argv         004233b8     nessus:nessus.dll
 0002:000003bc       __imp__nessuslib_version   004233bc     nessus:nessus.dll
 0002:000003c0       __imp__pty_logger          004233c0     nessus:nessus.dll
 0002:000003c4       __imp__arg_dup             004233c4     nessus:nessus.dll
 0002:000003c8       __imp__harg_close          004233c8     nessus:nessus.dll
 0002:000003cc       __imp__harg_walk_init      004233cc     nessus:nessus.dll
 0002:000003d0       __imp__arg_free_all        004233d0     nessus:nessus.dll
 0002:000003d4       __imp__harg_walk_next      004233d4     nessus:nessus.dll
 0002:000003d8       \177nessus_NULL_THUNK_DATA 004233d8     nessus:nessus.dll
 0002:000003dc       __imp__io_thtrp            004233dc     peks:peks.dll
 0002:000003e0       __imp__io_ctrl             004233e0     peks:peks.dll
 0002:000003e4       __imp____peks_nt_fprintf   004233e4     peks:peks.dll
 0002:000003e8       __imp__peks_strerr         004233e8     peks:peks.dll
 0002:000003ec       __imp__client_negotiate_session_key 004233ec     peks:peks.dll
 0002:000003f0       __imp__io_shutdown         004233f0     peks:peks.dll
 0002:000003f4       __imp__peks_client_authenticate 004233f4     peks:peks.dll
 0002:000003f8       __imp__peks_set_keep_alive_notice 004233f8     peks:peks.dll
 0002:000003fc       __imp____peks_nt_printf    004233fc     peks:peks.dll
 0002:00000400       __imp____peks_nt_setconsole 00423400     peks:peks.dll
 0002:00000404       __imp__peks_version        00423404     peks:peks.dll
 0002:00000408       __imp__peks_set_uservar    00423408     peks:peks.dll
 0002:0000040c       __imp__peks_set_homevar    0042340c     peks:peks.dll
 0002:00000410       __imp__peks_get_username   00423410     peks:peks.dll
 0002:00000414       __imp____peks_nt_exit      00423414     peks:peks.dll
 0002:00000418       __imp__peks_save_public_key 00423418     peks:peks.dll
 0002:0000041c       __imp__peks_delete_userkey 0042341c     peks:peks.dll
 0002:00000420       __imp__peks_list_keyfile   00423420     peks:peks.dll
 0002:00000424       __imp__peks_delete_hostkey 00423424     peks:peks.dll
 0002:00000428       __imp____peks_nt_getpass   00423428     peks:peks.dll
 0002:0000042c       __imp__peks_save_private_key 0042342c     peks:peks.dll
 0002:00000430       __imp__peks_private_key    00423430     peks:peks.dll
 0002:00000434       __imp__xfree               00423434     peks:peks.dll
 0002:00000438       __imp__pmalloc             00423438     peks:peks.dll
 0002:0000043c       __imp__peks_get_homedir    0042343c     peks:peks.dll
 0002:00000440       __imp____peks_nt_fopen     00423440     peks:peks.dll
 0002:00000444       __imp__peks_get_dirfile    00423444     peks:peks.dll
 0002:00000448       __imp____peks_nt_fgets     00423448     peks:peks.dll
 0002:0000044c       __imp__io_close            0042344c     peks:peks.dll
 0002:00000450       __imp____peks_nt_read      00423450     peks:peks.dll
 0002:00000454       __imp____peks_nt_open      00423454     peks:peks.dll
 0002:00000458       __imp____peks_nt_close     00423458     peks:peks.dll
 0002:0000045c       __imp__find_classes_by_name 0042345c     peks:peks.dll
 0002:00000460       __imp__io_recv             00423460     peks:peks.dll
 0002:00000464       __imp__io_send             00423464     peks:peks.dll
 0002:00000468       \177peks_NULL_THUNK_DATA   00423468     peks:peks.dll
 0002:00000470       __real@8@00000000000000000000 00423470     monitor_dialog.obj
 0002:00000478       __real@4@3fff8000000000000000 00423478     monitor_dialog.obj
 0002:0000047c       __real@4@4005c800000000000000 0042347c     html_graph_output.obj
 0002:00000480       __real@4@00000000000000000000 00423480     html_graph_output.obj
 0002:00000488       __real@8@40008000000000000000 00423488     price_conv.obj
 0002:00000490       __real@8@3ffe8000000000000000 00423490     price_conv.obj
 0002:00000498       __real@4@3ffe8000000000000000 00423498     price_conv.obj
 0002:000004a0       __real@8@3ff68000000000000000 004234a0     price_conv.obj
 0002:000004a8       __real@4@40078000000000000000 004234a8     price_conv.obj
 0002:000004b0       __real@8@3feea7c5ac471b478800 004234b0     gdc_pie.obj
 0002:000004b8       __real@8@bfeea7c5ac471b478800 004234b8     gdc_pie.obj
 0002:000004c0       __real@8@3ffec000000000000000 004234c0     gdc_pie.obj
 0002:000004c8       __real@8@4004e52ee0d31e0fc000 004234c8     gdc_pie.obj
 0002:000004d0       __real@8@4000c90fdaa22168c000 004234d0     gdc_pie.obj
 0002:000004d8       __real@8@400196cbe3f9990e9000 004234d8     gdc_pie.obj
 0002:000004e0       __real@8@4001c90fdaa22168c000 004234e0     gdc_pie.obj
 0002:000004e8       __real@8@3fffc90fdaa22168c000 004234e8     gdc_pie.obj
 0002:000004f0       __real@8@3ff98efa351294e9c800 004234f0     gdc_pie.obj
 0002:000004f8       __real@8@3ff8a3d70a3d70a3d800 004234f8     gdc_pie.obj
 0002:00000500       __real@8@4005c800000000000000 00423500     gdc_pie.obj
 0002:00000508       __real@4@407effffff0000000000 00423508     gdchart.obj
 0002:00000510       __real@8@3fff8000000000000000 00423510     gdchart.obj
 0002:00000518       __real@4@3ff98000000000000000 00423518     gdchart.obj
 0002:0000051c       __real@4@c07effffff0000000000 0042351c     gdchart.obj
 0002:0000052c       __IMPORT_DESCRIPTOR_nessus 0042352c     nessus:nessus.dll
 0002:00000540       __IMPORT_DESCRIPTOR_peks   00423540     peks:peks.dll
 0002:00000554       __IMPORT_DESCRIPTOR_gtk-1.3 00423554     gtk-1.3:gtk-1.3.dll
 0002:00000568       __IMPORT_DESCRIPTOR_gdk-1.3 00423568     gdk-1.3:gdk-1.3.dll
 0002:0000057c       __IMPORT_DESCRIPTOR_glib-1.3 0042357c     glib-1.3:glib-1.3.dll
 0002:00000590       __IMPORT_DESCRIPTOR_WSOCK32 00423590     wsock32:WSOCK32.dll
 0002:000005a4       __IMPORT_DESCRIPTOR_MSVCRT 004235a4     MSVCRT:MSVCRT.dll
 0002:000005b8       __IMPORT_DESCRIPTOR_KERNEL32 004235b8     kernel32:KERNEL32.dll
 0002:000005cc       __NULL_IMPORT_DESCRIPTOR   004235cc     nessus:nessus.dll
 0003:00000000       ___xc_a                    00425000     MSVCRT:cinitexe.obj
 0003:00000004       ___xc_z                    00425004     MSVCRT:cinitexe.obj
 0003:00000008       ___xi_a                    00425008     MSVCRT:cinitexe.obj
 0003:0000000c       ___xi_z                    0042500c     MSVCRT:cinitexe.obj
 0003:00009f98       _peks_get_pwd              0042ef98     nessus.obj
 0003:00009f9c       _keylen                    0042ef9c     nessus.obj
 0003:00009fa0       _kf                        0042efa0     nessus.obj
 0003:0005ea64       _GDC_generate_gif          00483a64     html_graph_output.obj
 0003:0005ea68       _GDC_title_size            00483a68     html_graph_output.obj
 0003:0005ea6c       _GDC_ytitle_size           00483a6c     html_graph_output.obj
 0003:0005ea70       _GDC_xtitle_size           00483a70     html_graph_output.obj
 0003:0005ea74       _GDC_yaxisfont_size        00483a74     html_graph_output.obj
 0003:0005ea78       _GDC_xaxisfont_size        00483a78     html_graph_output.obj
 0003:0005ea7c       _GDC_xlabel_spacing        00483a7c     html_graph_output.obj
 0003:0005ea7e       _GDC_ylabel_density        00483a7e     html_graph_output.obj
 0003:0005ea80       _GDC_requested_ymin        00483a80     html_graph_output.obj
 0003:0005ea84       _GDC_requested_ymax        00483a84     html_graph_output.obj
 0003:0005ea88       _GDC_requested_yinterval   00483a88     html_graph_output.obj
 0003:0005ea8c       _GDC_0Shelf                00483a8c     html_graph_output.obj
 0003:0005ea8d       _GDC_grid                  00483a8d     html_graph_output.obj
 0003:0005ea8e       _GDC_xaxis                 00483a8e     html_graph_output.obj
 0003:0005ea8f       _GDC_yaxis                 00483a8f     html_graph_output.obj
 0003:0005ea90       _GDC_yaxis2                00483a90     html_graph_output.obj
 0003:0005ea91       _GDC_yval_style            00483a91     html_graph_output.obj
 0003:0005ea94       _GDC_3d_depth              00483a94     html_graph_output.obj
 0003:0005ea98       _GDC_3d_angle              00483a98     html_graph_output.obj
 0003:0005ea99       _GDC_bar_width             00483a99     html_graph_output.obj
 0003:0005ea9c       _GDC_HLC_style             00483a9c     html_graph_output.obj
 0003:0005eaa0       _GDC_HLC_cap_width         00483aa0     html_graph_output.obj
 0003:0005eaa4       _GDC_annotation_font       00483aa4     html_graph_output.obj
 0003:0005eaa8       _GDC_thumbval              00483aa8     html_graph_output.obj
 0003:0005eaac       _GDC_border                00483aac     html_graph_output.obj
 0003:0005eab0       _GDC_GridColor             00483ab0     html_graph_output.obj
 0003:0005eab4       _GDC_LineColor             00483ab4     html_graph_output.obj
 0003:0005eab8       _GDC_PlotColor             00483ab8     html_graph_output.obj
 0003:0005eabc       _GDC_VolColor              00483abc     html_graph_output.obj
 0003:0005eac0       _GDC_TitleColor            00483ac0     html_graph_output.obj
 0003:0005eac4       _GDC_XTitleColor           00483ac4     html_graph_output.obj
 0003:0005eac8       _GDC_YTitleColor           00483ac8     html_graph_output.obj
 0003:0005eacc       _GDC_YTitle2Color          00483acc     html_graph_output.obj
 0003:0005ead0       _GDC_XLabelColor           00483ad0     html_graph_output.obj
 0003:0005ead4       _GDC_YLabelColor           00483ad4     html_graph_output.obj
 0003:0005ead8       _GDC_YLabel2Color          00483ad8     html_graph_output.obj
 0003:0005eadc       _GDCPIE_PlotColor          00483adc     html_graph_output.obj
 0003:0005eae0       _GDCPIE_LineColor          00483ae0     html_graph_output.obj
 0003:0005eae4       _GDCPIE_EdgeColor          00483ae4     html_graph_output.obj
 0003:0005eae8       _GDCPIE_other_threshold    00483ae8     html_graph_output.obj
 0003:0005eaea       _GDCPIE_3d_angle           00483aea     html_graph_output.obj
 0003:0005eaec       _GDCPIE_3d_depth           00483aec     html_graph_output.obj
 0003:0005eaf0       _GDCPIE_title_size         00483af0     html_graph_output.obj
 0003:0005eaf4       _GDCPIE_label_size         00483af4     html_graph_output.obj
 0003:0005eaf8       _GDCPIE_label_dist         00483af8     html_graph_output.obj
 0003:00079058       _GDC_fontc                 0049e058     gdc.obj
 0003:00079130       _cost                      0049e130     gd.obj
 0003:000796d0       _sint                      0049e6d0     gd.obj
 0003:00079eb0       _gdFontTinyData            0049eeb0     gdfontt.obj
 0003:0007c6b0       _gdFontTinyRep             004a16b0     gdfontt.obj
 0003:0007c6c4       _gdFontTiny                004a16c4     gdfontt.obj
 0003:0007c6c8       _gdFontSmallData           004a16c8     gdfonts.obj
 0003:000814c8       _gdFontSmallRep            004a64c8     gdfonts.obj
 0003:000814dc       _gdFontSmall               004a64dc     gdfonts.obj
 0003:000814e0       _gdFontMediumBoldData      004a64e0     gdfontmb.obj
 0003:00086fe0       _gdFontMediumBoldRep       004abfe0     gdfontmb.obj
 0003:00086ff4       _gdFontMediumBold          004abff4     gdfontmb.obj
 0003:00086ff8       _gdFontLargeData           004abff8     gdfontl.obj
 0003:0008eff8       _gdFontLargeRep            004b3ff8     gdfontl.obj
 0003:0008f00c       _gdFontLarge               004b400c     gdfontl.obj
 0003:0008f010       _gdFontGiantData           004b4010     gdfontg.obj
 0003:00097710       _gdFontGiantRep            004bc710     gdfontg.obj
 0003:00097724       _gdFontGiant               004bc724     gdfontg.obj
 0003:00097730       ___defaultmatherr          004bc730     MSVCRT:merr.obj
 0003:0009773c       _Plugins                   004bc73c     nessus.obj
 0003:00097740       _Scanners                  004bc740     nessus.obj
 0003:00097744       _Alt_rcfile                004bc744     nessus.obj
 0003:00097748       _stored_pwd                004bc748     nessus.obj
 0003:0009774c       _First_time                004bc74c     nessus.obj
 0003:00097750       _key                       004bc750     nessus.obj
 0003:00097788       _splash_screen             004bc788     splash_screen.obj
 0003:00097794       _GDC_hold_img              004bc794     html_graph_output.obj
 0003:00097798       _GDC_image                 004bc798     html_graph_output.obj
 0003:0009779c       _GDC_ylabel_fmt            004bc79c     html_graph_output.obj
 0003:000977a0       _GDC_ylabel2_fmt           004bc7a0     html_graph_output.obj
 0003:000977a4       _GDC_stack_type            004bc7a4     html_graph_output.obj
 0003:000977a8       _GDC_annotation            004bc7a8     html_graph_output.obj
 0003:000977ac       _GDC_num_scatter_pts       004bc7ac     html_graph_output.obj
 0003:000977b0       _GDC_scatter               004bc7b0     html_graph_output.obj
 0003:000977b4       _GDC_thumbnail             004bc7b4     html_graph_output.obj
 0003:000977b8       _GDC_BGColor               004bc7b8     html_graph_output.obj
 0003:000977bc       _GDC_ExtVolColor           004bc7bc     html_graph_output.obj
 0003:000977c0       _GDC_SetColor              004bc7c0     html_graph_output.obj
 0003:000977c4       _GDC_ExtColor              004bc7c4     html_graph_output.obj
 0003:000977c8       _GDC_transparent_bg        004bc7c8     html_graph_output.obj
 0003:000977cc       _GDC_BGImage               004bc7cc     html_graph_output.obj
 0003:000977d0       _GDC_hard_size             004bc7d0     html_graph_output.obj
 0003:000977d4       _GDC_hard_xorig            004bc7d4     html_graph_output.obj
 0003:000977d8       _GDC_hard_graphwidth       004bc7d8     html_graph_output.obj
 0003:000977dc       _GDC_hard_yorig            004bc7dc     html_graph_output.obj
 0003:000977e0       _GDC_hard_grapheight       004bc7e0     html_graph_output.obj
 0003:000977e4       _GDCPIE_BGColor            004bc7e4     html_graph_output.obj
 0003:000977e8       _GDCPIE_title              004bc7e8     html_graph_output.obj
 0003:000977ec       _GDCPIE_label_line         004bc7ec     html_graph_output.obj
 0003:000977f0       _GDCPIE_explode            004bc7f0     html_graph_output.obj
 0003:000977f4       _GDCPIE_Color              004bc7f4     html_graph_output.obj
 0003:000977f8       _GDCPIE_missing            004bc7f8     html_graph_output.obj
 0003:000977fc       _GDCPIE_percent_labels     004bc7fc     html_graph_output.obj
 0003:000a7fa8       __dowildcard               004ccfa8     MSVCRT:wildcard.obj
 0003:000a7fac       __newmode                  004ccfac     MSVCRT:_newmode.obj
 0003:000a7fb0       __commode                  004ccfb0     MSVCRT:xncommod.obj
 0003:000a7fb4       __fmode                    004ccfb4     MSVCRT:xtxtmode.obj
 0003:000a7fb8       _ZeroDataBlock             004ccfb8     <common>
 0003:000a7fbc       _GDC_title                 004ccfbc     <common>
 0003:000a7fc0       _GDC_xtitle                004ccfc0     <common>
 0003:000a7fc4       _GDC_ytitle                004ccfc4     <common>
 0003:000a7fc8       _GDC_ytitle2               004ccfc8     <common>
 0003:000a7fcc       _ScannersNum               004ccfcc     <common>
 0003:000a7fd0       _F_nessusd_running         004ccfd0     <common>
 0003:000a7fd4       _ArgSock                   004ccfd4     <common>
 0003:000a7fd8       _MainDialog                004ccfd8     <common>
 0003:000a7fdc       _PluginsNum                004ccfdc     <common>
 0003:000a7fe0       _F_quiet_mode              004ccfe0     <common>
 0003:000a7fe4       _F_show_pixmaps            004ccfe4     <common>
 0003:000a7fe8       _Prefs                     004ccfe8     <common>
 0003:000a7fec       _GlobalSocket              004ccfec     <common>
 0003:000a7ff0       ___onexitend               004ccff0     <common>
 0003:000a7ff4       ___onexitbegin             004ccff4     <common>
 0003:000a7ff8       __adjust_fdiv              004ccff8     <common>

 entry point at        0001:000213bc

 Static symbols

 0001:0001dc90       _gdImageBrushApply         0041ec90 f   gd.obj
 0001:0001dd60       _gdImageTileApply          0041ed60 f   gd.obj
 0001:0001e220       _dashedSet                 0041f220 f   gd.obj
 0001:0001e570       _strlen16                  0041f570 f   gd.obj
 0001:0001ea30       _colorstobpp               0041fa30 f   gd.obj
 0001:0001eaa0       _GIFEncode                 0041faa0 f   gd.obj
 0001:0001ec50       _Putword                   0041fc50 f   gd.obj
 0001:0001ec90       _compress                  0041fc90 f   gd.obj
 0001:0001ed90       _GIFNextPixel              0041fd90 f   gd.obj
 0001:0001edd0       _BumpPixel                 0041fdd0 f   gd.obj
 0001:0001eeb0       _output                    0041feb0 f   gd.obj
 0001:0001ef10       _block_out                 0041ff10 f   gd.obj
 0001:0001ef40       _write_block               0041ff40 f   gd.obj
 0001:0001ef80       _output_flush              0041ff80 f   gd.obj
 0001:0001efa0       _block_flush               0041ffa0 f   gd.obj
 0001:0001efb0       _did_clear                 0041ffb0 f   gd.obj
 0001:0001eff0       _rl_flush                  0041fff0 f   gd.obj
 0001:0001f080       _output_plain              00420080 f   gd.obj
 0001:0001f0f0       _rl_flush_fromclear        004200f0 f   gd.obj
 0001:0001f1b0       _max_out_clear             004201b0 f   gd.obj
 0001:0001f1c0       _reset_out_clear           004201c0 f   gd.obj
 0001:0001f1f0       _rl_flush_clearorrep       004201f0 f   gd.obj
 0001:0001f240       _compute_triangle_count    00420240 f   gd.obj
 0001:0001f2b0       _isqrt                     004202b0 f   gd.obj
 0001:0001f2f0       _rl_flush_withtable        004202f0 f   gd.obj
 0001:0001f400       _init_statics              00420400 f   gd.obj
 0001:0001f720       _ReadColorMap              00420720 f   gd.obj
 0001:0001f790       _DoExtension               00420790 f   gd.obj
 0001:0001f850       _GetDataBlock              00420850 f   gd.obj
 0001:0001f870       _GetDataBlock_             00420870 f   gd.obj
 0001:0001f8e0       _ReadImage                 004208e0 f   gd.obj
 0001:0001fac0       _LWZReadByte               00420ac0 f   gd.obj
 0001:0001fae0       _LWZReadByte_              00420ae0 f   gd.obj
 0001:0001fe50       _GetCode                   00420e50 f   gd.obj
 0001:0001fe70       _GetCode_                  00420e70 f   gd.obj
 0001:00017d10       _qcmpr                     00418d10 f   gdchart.obj
 0001:0001d8c0       _barcmpr                   0041e8c0 f   gdchart.obj
 0001:00017330       _ocmpr                     00418330 f   gdc_pie.obj
 0001:000130f0       _disable_all               004140f0 f   prefs_plugins.obj
 0001:000131d0       _enable_all                004141d0 f   prefs_plugins.obj
 0001:000132b0       _enable_all_but_dos        004142b0 f   prefs_plugins.obj
 0001:000133b0       _prefs_plugin_list_callback 004143b0 f   prefs_plugins.obj
 0001:00013420       _prefs_family_list_callback 00414420 f   prefs_plugins.obj
 0001:00013850       _warning_sign              00414850 f   prefs_plugins.obj
 0001:00013910       _warning_expl              00414910 f   prefs_plugins.obj
 0001:00013930       _prefs_plugin_list_toggle_callback 00414930 f   prefs_plugins.obj
 0001:00013cf0       _prefs_family_toggle_callback 00414cf0 f   prefs_plugins.obj
 0001:00012880       _dialog_change_passphrase  00413880 f   prefs_dialog_user.obj
 0001:00012910       _dialog_keyring            00413910 f   prefs_dialog_user.obj
 0001:00012950       _keyring_peks_callback     00413950 f   prefs_dialog_user.obj
 0001:00012a30       _sigh_button_event         00413a30 f   prefs_dialog_user.obj
 0001:00012af0       _add_rule_callback         00413af0 f   prefs_dialog_user.obj
 0001:00012210       _prefs_scanner_list_toggle_callback 00413210 f   prefs_dialog_scan_opt.obj
 0001:00012290       _scanner_infos_cb          00413290 f   prefs_dialog_scan_opt.obj
 0001:00011540       _pprefs_add_separator      00412540 f   prefs_dialog_plugins_prefs.obj
 0001:00011600       _pprefs_add_entry          00412600 f   prefs_dialog_plugins_prefs.obj
 0001:00011770       _pprefs_add_radio          00412770 f   prefs_dialog_plugins_prefs.obj
 0001:00011a00       _pprefs_add_checkbox       00412a00 f   prefs_dialog_plugins_prefs.obj
 0001:00010b70       _get_username              00411b70 f   prefs_dialog_auth.obj
 0001:00010b90       _prefs_dialog_logout_callback 00411b90 f   prefs_dialog_auth.obj
 0001:00010c00       _prefs_dialog_login_callback 00411c00 f   prefs_dialog_auth.obj
 0001:0000fa80       _prefs_dialog_set_tooltips 00410a80 f   prefs_dialog.obj
 0001:0000e970       _parse_portname            0040f970 f   xml_output.obj
 0001:0000e270       _cli_test_monitor          0040f270 f   cli.obj
 0001:0000c170       _make_index                0040d170 f   html_graph_output.obj
 0001:0000c9f0       _insert_img                0040d9f0 f   html_graph_output.obj
 0001:0000ca10       _risk_severity             0040da10 f   html_graph_output.obj
 0001:0000cb20       _complete                  0040db20 f   html_graph_output.obj
 0001:0000cb60       _risk_severity_by_host     0040db60 f   html_graph_output.obj
 0001:0000cb90       _risk_severity_by_port     0040db90 f   html_graph_output.obj
 0001:0000cc20       _risk_severity_by_kind     0040dc20 f   html_graph_output.obj
 0001:0000cd10       _strcasestr                0040dd10 f   html_graph_output.obj
 0001:0000cd70       _most_vulnerable_services  0040dd70 f   html_graph_output.obj
 0001:0000cdb0       _fill_list_of_services     0040ddb0 f   html_graph_output.obj
 0001:0000ce10       _fill_list_of_services_by_ports 0040de10 f   html_graph_output.obj
 0001:0000cea0       _top_n_most_vulnerable_services 0040dea0 f   html_graph_output.obj
 0001:0000cf90       _most_present_services     0040df90 f   html_graph_output.obj
 0001:0000cfd0       _fill_list_of_services_presence 0040dfd0 f   html_graph_output.obj
 0001:0000d030       _fill_list_of_services_presence_by_ports 0040e030 f   html_graph_output.obj
 0001:0000d090       _top_n_most_present_services 0040e090 f   html_graph_output.obj
 0001:0000d180       _most_used_operating_systems 0040e180 f   html_graph_output.obj
 0001:0000d1c0       _fill_operating_systems_list 0040e1c0 f   html_graph_output.obj
 0001:0000d2b0       _top_n_operating_systems   0040e2b0 f   html_graph_output.obj
 0001:0000d3a0       _create_host_report        0040e3a0 f   html_graph_output.obj
 0001:0000d6f0       _host_details              0040e6f0 f   html_graph_output.obj
 0001:0000dcb0       _print_data_with_cve_link  0040ecb0 f   html_graph_output.obj
 0001:0000dd90       _convert_cr_to_html        0040ed90 f   html_graph_output.obj
 0001:0000de30       _portname_to_ahref         0040ee30 f   html_graph_output.obj
 0001:0000b530       _splash_setup_passphrase   0040c530 f   splash_screen.obj
 0001:0000b590       _splash_setup_passphrase_build 0040c590 f   splash_screen.obj
 0001:0000bb70       _splash_setup_passphrase_cancel 0040cb70 f   splash_screen.obj
 0001:0000bbe0       _splash_setup_passphrase_ok 0040cbe0 f   splash_screen.obj
 0001:0000bea0       _splash_init               0040cea0 f   splash_screen.obj
 0001:0000b070       _printf_line               0040c070 f   text_output.obj
 0001:0000a460       _print_data_with_cve_link  0040b460 f   html_output.obj
 0001:0000a540       _convert_cr_to_html        0040b540 f   html_output.obj
 0001:0000a5e0       _portname_to_ahref         0040b5e0 f   html_output.obj
 0001:00009ab0       _sub_most_dangerous_host_holes 0040aab0 f   report_utils.obj
 0001:00009b00       _sub_most_dangerous_host_warnings 0040ab00 f   report_utils.obj
 0001:00009b50       _sub_most_dangerous_host_notes 0040ab50 f   report_utils.obj
 0001:00009250       _latex_report_category     0040a250 f   latex_output.obj
 0001:000092d0       _latex_print_header        0040a2d0 f   latex_output.obj
 0001:00009370       _latex_print_footer        0040a370 f   latex_output.obj
 0001:00006b90       _findings_to_tree          00407b90 f   report.obj
 0001:00006e20       _data_to_tree              00407e20 f   report.obj
 0001:00006f20       _data_to_tree_build_label  00407f20 f   report.obj
 0001:00006f80       _findings_to_tree_build_label 00407f80 f   report.obj
 0001:00006fe0       _report_build_label        00407fe0 f   report.obj
 0001:000071b0       _create_report_window      004081b0 f   report.obj
 0001:000071d0       _do_create_report_window   004081d0 f   report.obj
 0001:00007870       _fill_summary_box          00408870 f   report.obj
 0001:00007cd0       _report_click              00408cd0 f   report.obj
 0001:00007ea0       _summary_host_label        00408ea0 f   report.obj
 0001:00007f80       _create_report_window_by_port 00408f80 f   report.obj
 0001:00008160       _save_report_ask           00409160 f   report.obj
 0001:00008480       _save_report               00409480 f   report.obj
 0001:000069f0       _target_file_apply         004079f0 f   read_target_file.obj
 0001:000059e0       _preferences_get_filename  004069e0 f   preferences.obj
 0001:00005d20       _preferences_new           00406d20 f   preferences.obj
 0001:00005df0       _prefs_add_subcategory     00406df0 f   preferences.obj
 0001:00005ed0       _prefs_buffer_parse        00406ed0 f   preferences.obj
 0001:00006510       _new_pluginset             00407510 f   preferences.obj
 0001:00004f10       _pass_build_dialog         00405f10 f   password_dialog.obj
 0001:00005250       _pass_dialog_callback      00406250 f   password_dialog.obj
 0001:000048e0       _client_save_hole          004058e0 f   parser.obj
 0001:00004a10       _client_save_info          00405a10 f   parser.obj
 0001:00004b40       _client_save_note          00405b40 f   parser.obj
 0001:00004d80       _add_port                  00405d80 f   parser.obj
 0001:00003a90       _key_initialization_stuff  00404a90 f   nessus.obj
 0001:00003d50       _action_header             00404d50 f   nessus.obj
 0001:00003d70       _version_check             00404d70 f   nessus.obj
 0001:00001ef0       _idle_socket               00402ef0 f   monitor_dialog.obj
 0001:000020f0       _monitor_stop_whole_test_destroy 004030f0 f   monitor_dialog.obj
 0001:00002100       _monitor_stop_whole_test   00403100 f   monitor_dialog.obj
 0001:00002170       _monitor_input_callback    00403170 f   monitor_dialog.obj
 0001:00002390       _monitor_list_update       00403390 f   monitor_dialog.obj
 0001:000026c0       _label_name                004036c0 f   monitor_dialog.obj
 0001:000027d0       _monitor_add_host          004037d0 f   monitor_dialog.obj
 0001:00002d80       _monitor_stop_test         00403d80 f   monitor_dialog.obj
 0001:00002da0       _build_plugins_order_table 00403da0 f   monitor_dialog.obj
 0001:000019e0       _show_dialog_and_wait_cb   004029e0 f   error_dialog.obj
 0001:000001c0       _setup_plug_list           004011c0 f   attack.obj
